:030000000219FDE5
:03000B000200AA46
:03002B0002016669
:03005B000202F9A5
:030073000202DFA7
:1000800002030406080C10182030406080040608A3
:100090000C10182030406080A0C000070F1F3F0DDB
:1000A0000D04050D050305030302C2AFC0D0C0E077
:1000B000206217E5256002E473E525F4F58A758B67
:1000C00000D262D0E0D0D0D2AF3285268AC262E5BB
:1000D00026F46036306803207210758B00D0E0D0B3
:1000E000D0C290C291C292D2AF32C290C291C2929B
:1000F000206E0D20660A7401D5E0FDE57EF4529075
:10010000758B00D0E0D0D0D2AF32758A00C28DD2CC
:1001100062210001B9306805206602D29001B93031
:100120006805206602D29101B9306805206602D2C6
:100130009201B9D29330680A2066077405D5E0FDB4
:10014000D29001B9D29430680A2066077405D5E0D0
:10015000FDD29101B9D29530680A2066077405D5A1
:10016000E0FDD29201B9C2AFC2AD53E6EFC0D0C03C
:10017000E0D2D3D2AFC2CEE52A6007207449152A57
:1001800021C77800790020742EE580307E01F4309C
:10019000E70278FF53DACF207E0343DA20307E0374
:1001A00043DA10C2D8C271E580307E01F430E70234
:1001B00079FFC3E89970CB306103752A1820740366
:1001C000752A18885FD27020740DE52B6004152BFA
:1001D00021D743DA01C2D82070024135A85F2061DF
:1001E00002C2702074367982B70431C3E894F040BB
:1001F0000374F0F8E8C4540F28F87984B703024177
:100200001CC313C3138721200802C313200A06C38B
:10021000C898F8411C28F8500374FFF88822E52D8F
:1002200054066011E533C313C31324062522F522B7
:1002300050037522FF7882B60459852224A824C36E
:10024000E52495644002A864C3E895664002A86668
:100250008825E56970024186C3E8AA699A5003E8D7
:10026000FAE4F9EAC333FBE56BF45B29400D256A38
:10027000F8E56A6002156A400B41860AC3E56A9A8E
:100280005002056A78FF8826C26EC3E52694F840BE
:1002900002D26EC3E52594404002D26420CF0AD03A
:1002A000E0D0D043E610D2AD32C2CF053A7801E5B6
:1002B0002A6005307402152AC3E55F940140057574
:1002C000620041D5756300756C00E5622401F5623A
:1002D00050037562FFD0E0D0D043E610D2AD32C2F9
:1002E000AFC0D053E67FC2607591008556948557A4
:1002F00095759104D0D0D2AF32C2AF53E6EFC2AD04
:10030000C0D0C0E0C0F0D2D3D2AFA8FBA9FCC2D805
:10031000307102616053DACF207E0343DA10307E01
:100320000343DA20D271E580307E01F420E70261D8
:100330003788278928A18753DACF207E0343DA2024
:10034000307E0343DA10C2D8C271307402A17378D0
:1003500000E580307E01F430E702A173885FA15B85
:1003600053DACF207E0343DA20307E0343DA10C213
:1003700071206102813953DACF207E0343DA1030D5
:100380007E0343DA20C2D8D271885A895BC3E895CC
:1003900058F8E99559F97B007E087A00C3E8948CF7
:1003A000E994005005755E00812B882178A2E6A8AB
:1003B000216055C3E894C8E994005008E4D2E4FBF6
:1003C0007A0A8106C3E89468E994015008E4D2E30C
:1003D000FB7A0F8106C3E894D0E994025008E4D276
:1003E000E2FB7A1E8106C3E894A0E994055008E474
:1003F000D2E1FB7A3C8106C3E89498E9940850085E
:10040000E4D2E0FB7A787E00C3E8955CFCE9955D78
:10041000FD30E70AECF42401FCEDF43400FD755ED8
:1004200000C3EC9AED9E5003755E01885C895D8582
:100430005A58855B597802A15BC3E89527F8E9957E
:1004400028F9307C02A13F307B02A13F307A02A123
:1004500038207502815CE9FDE8FC817BE9C313F972
:10046000E813F8307902A138E9C313F9E813F8303A
:0F0470007802A138E9C313FDE813FC206126C30D
:10047F00EC941CED940240028192ED7018C3EC9441
:10048F00C850120529C3E529940A5002A173755F5C
:10049F0000D270A173E529600215297888E6F974F6
:1004AF0000207F087896B90302789EE624FAFEE4CE
:1004BF003400FFC3EC9EFCED9FFD9208B90310A220
:1004CF00085007207609D27681DE307602C276A2F6
:1004DF00085016B9030DECF42401FCEDF43400FDC3
:1004EF000204F878007900A13FB90315EC33FCED55
:1004FF0033FDC3EC940AFCED9400FD50047C007DA9
:10050F0000C3EC94FFED9400400678FF7900A13F03
:10051F00EC8575F0A4C5F0A2F733F879004003021B
:10052F00055B78FF790002055BE9C313F9E813F85F
:10053F00307C0EE9600278FFC3E81338F8E434002A
:10054F00F9C3E894FFE99400400278FF885FD27006
:10055F00206102A173741FF4552F4BF52FC274EB5A
:10056F007002D274752A18307403752A0A3061022A
:10057F00A18720740353DAFE207403752B06D0F085
:10058F00D0E0D0D0D2AD43E6103279010205B77971
:10059F00030205B7790A0205B7791E0205B7796418
:1005AF000205B779C80205B77817E4D5E0FDD8FA88
:1005BF00D9F6227A147B780205DE7A107B8C02053D
:1005CF00DE7A0D7BB40205DE7A0B7BC80205DE797D
:1005DF0002B27DE4D294D5E0FDD291D5E0FDC29177
:1005EF00D5E0FDC294D5E0FDD290E576D5E0FDC211
:1005FF00907496D5E0FDD9D9EAF8D5E0FDD8FBDBAC
:10060F00CED29422C37C007D0075F00005F0EA3352
:10061F00FAEB33FB50F6EB13FBEA13FAC3E9FFE8EF
:10062F00FEE89AF8E99BF95004EFF9EEF8B3EC33D2
:10063F00FCED33FDD5F0DFEDF9ECF822E889F08A17
:10064F0020D2D4F8A9F07B0030F70B7BFFF4240104
:10065F00F8E9F43400F9E88520F0A4ADF0F8E98565
:10066F0020F0A4AFF0FEED2EF974003FFA7C04C326
:10067F00EA13FAE913F9E813F8DCF48BF030F70A10
:10068F00E8F42401F8E9F43400F9E889F0C2D4F869
:10069F00A9F0227882B604030206FDC3E55F940138
:1006AF0040030206C7852224E4F545F546F547F5D4
:1006BF0048F549C26D0206FD7882E6FCD26DE5224F
:1006CF00F523783879C7AA40AB41C3EB13FBEA1384
:1006DF00FAEC146013C3EB13FBEA13FAEC14146077
:1006EF0007C3EB13FBEA13FAD1138845894622C3DC
:1006FF00E5459523F8E5469400F9500CC3E894803E
:10070F00E994FF401602072EC3E8947FE994005046
:10071F000302072E787F790002072E788079FF88F1
:10072F004A894B22E54A2547F8E54B3548F9854B71
:10073F0020E4300701F43549FA30E709C3EA94F0B1
:10074F00401502076CC3EA940F500302076C78FF41
:10075F0079FF7A0F02076C780079007AF0C3E524ED
:10076F009564500AC374019524500B02078AE54B18
:10077F0020E70E02078AE54B30E706884789488A4B
:10078F00492278A4E6FAC3E54A33F8E54B33F9D1A9
:10079F004BE930E70BC3E89480E994FF4013E1C4C1
:1007AF00C3E8947FE994005002E1C4787F7900E1B7
:1007BF00C4788079FFE820E715C3E52398F840094E
:1007CF00C3E8940140030207EB78010207EBE8F45A
:1007DF0024012523F840030207EB78FF884C227889
:1007EF00A5E6FAA848A949D14BE930E70CC3E8942C
:1007FF0001E994FF401602081FC3E894FFE9940033
:10080F00500302081F78FF790002081F780179FF53
:10081F00E920E715C3E54C98F84009C3E894014077
:10082F00030208467801020846E8F42401254CF833
:10083F00400302084678FF88242278FFC2642069AB
:10084F003D206A12D264C3E541940A4009C3E525ED
:10085F0094405002C26479A1E76023E541601F74A0
:0F086F00FF8541F0848539F0306A0375F005A4E8
:10087E00F8C5F0600278FFC3E895675002A8678854
:10088E006622C3E5409440E5419401E566500314A9
:10089E0001A1046002F566220208A92275E89022E1
:1008AE007883E6FFE5E820ECF7A8BDA9BE0573C383
:1008BE00E57394084052757300E9FA79A0E7604435
:1008CE00EA7007E574601B0208E4C3E895746010D3
:1008DE00E5745006600C140208F00460F90208F08A
:1008EE00E574F574C394F6401B7564C0C39406405A
:1008FE0013756480C39406400B756440C394064020
:10090E000375640075BB0622E5642410500274FF63
:10091E00F5647982B70402213DC3A864E52498509A
:10092E0002A824C3E895664002A86688258826E5B5
:10093E0073B4070375BB1022743279A687F0A4C571
:10094E00F0A2F733F8C3E895644002A864882288C1
:10095E0024882588268867227540007541F022C2BA
:10096E00AF75C820A8CCA9CDAA3A30CF010A75C858
:10097E0024D2AFAB3BAC3C883B893CC3E89BF8E947
:10098E009C206908F9306702418221DFAD3D8A3D26
:10099E00F9EA9DFA600478FF79FFAE3EAF3F8B3ED9
:1009AE008C3FC3EC9FFCC3E99CF542A83BA93CC31A
:1009BE00E89EF8E99FF9C3E54113FBE54013FAE819
:1009CE002AF540E93BF54150067540FF7541FF4160
:1009DE0029AA40AB41AC40AD417E047F02C3EB94EB
:1009EE000440021E1FC3EB940840021E1FC3ED13EA
:1009FE00FDEC13FCDEF7C3EA9CFAEB9DFBEF6009FE
:100A0E00C3E913F9E813F8DFF7EA28FAEB39FB8AA2
:100A1E00408B4150067BFF8B408B41C3EB940250C1
:100A2E0002D2673069047F0341547892E6FFC3E532
:100A3E0037948240110FC3E53794A040010FC3EFE6
:100A4E00940640027F057E04E541C4540FF9E5414A
:100A5E00C454F0F8E540C4540F28F8C3E89EFAE9F0
:100A6E009400FB4009C3EA9402EB940050047A020E
:100A7E00E4FB41CEAA40AB41EBC4FEEAC4540F4E98
:100A8E00FCC3EA9CFAEB9400FBC3E813C313F8EA29
:100A9E0028FAEB3400FB8A408B41C3EB94024002F0
:100AAE00C2677804EBC4FE7B00EAC4540F4EFAC34F
:100ABE00EA98FA4005C3940250027A027892E6FF51
:100ACE0030600241CE855256855357D26043E68040
:100ADE00C3E49AF8E49BF93067026168E8FAE9FB2F
:100AEE00D3E913FDE813FC88528953C3EF940360D6
:100AFE0038EF20E00DE82CF8E93DF9ECFAEDFB02B9
:100B0E000B23E828F8E939F9C3E82402F8E93400A0
:100B1E00F97AFE7BFFC3EF9403400E8A548B5588FF
:100B2E004E894F8C508D51619C885489558A4E8BBD
:100B3E004F8C508D51306920C3E53394034019E535
:100B4E0042A2E713F8E555F4240138400B20E708DC
:100B5E007554FFF42401F555619CE8FAD3E813FCB3
:100B6E008852C3EF94036020EF20E007E82CF8ECE6
:100B7E00FA6188E8282402F87AFEC3EF940340084D
:100B8E008A54884E8C50619C88548A4E8C50E56BEA
:100B9E00C3335002646BF56B30600261A67534028C
:100BAE00D26043E680E52D54066026A840A941C3D5
:100BBE00E913F9E813F8C2AF53E67F759100C3E469
:100BCE0098F594E499F595759104D26043E680D238
:100BDE00AF22D265754400752000306B037520403E
:100BEE00020BFFD265754400752040306B037520F3
:100BFE0000D2AF7801206722E52D54066002C2654F
:100C0E00C3E5419405401378029405400878039497
:100C1E000540027806306902780A206019E54460C2
:100C2E001530690AC3E53394034003D53406D2AFB9
:100C3E00D26C81D171AED2AF0000C2AF206726E573
:100C4E0041C3FB940F40027B0FEB2405307301234D
:100C5E00306A02742820620123F93069027982E534
:0F0C6E008BC39940B50544E59BF45440B5200273
:100C7D0081BB30690A08C3E8940A40010881282025
:100C8D00650261FFC26553E67F759100306710758F
:100C9D0094007595FE759104D26043E68061FFAEB8
:100CAD0040AF41C3E49EF594E49FF59581A2C3E561
:100CBD00339402500261FF30650261FFD80281CF8B
:100CCD008128C26C53E67F759100855494855595A6
:100CDD00759104854E56854F57D26043E680D2AF4D
:100CED00E52D54066008206A020533020D0B306CA9
:100CFD000D206B0A20650715811581021576227866
:100D0D00003064053065027801E53775F007A4F908
:100D1D00E5F028F5F0E9A2F013A2F113A2F213F514
:100D2D0037C394785003753778C3E5379538400845
:100D3D00D266C290C291C292306002A145855056D2
:100D4D00855157D26043E68022207D11C2AF754395
:100D5D0002D294C293D2AF759F11020F25C2AF7507
:100D6D004302D294C295D2AF759F11020F253072F6
:100D7D0043207D20C2AF754303900144757E10C2A0
:100D8D0092D295306204D291A199C294D2AF759F3F
:100D9D0001020F25C2AF754303900144757E10C249
:100DAD0090D293306204D291A1B9C294D2AF759F03
:100DBD0021020F25207D17C2AF75430390011FC27D
:100DCD0092306202D291D2AF759F01020F25C2AF50
:100DDD0075430390011FC290306202D291D2AF755C
:100DED009F21020F25207D11C2AF754304D293C2FE
:100DFD0095D2AF759F21020F25C2AF754304D295D1
:100E0D00C293D2AF759F01020F25307243207D2012
:100E1D00C2AF754305900133757E08C291D29430EF
:100E2D006204D290C135C293D2AF759F11020F25C6
:100E3D00C2AF754305900155757E20C291D2943095
:100E4D006204D292C155C295D2AF759F11020F2582
:100E5D00207D17C2AF754305900115C29130620216
:100E6D00D290D2AF759F11020F25C2AF7543059079
:100E7D000129C2913062EBD292D2AF759F11020F50
:100E8D0025207D11C2AF754306D295C294D2AF75A0
:100E9D009F01020F25C2AF754306D293C294D2AF04
:100EAD00759F21020F25307242207D20C2AF754300
:100EBD0001900155757E20C290D293306204D2927A
:100ECD00C1D1C295D2AF759F21020F25C2AF754317
:100EDD0001900133757E08C292D295306204D29092
:100EED00C1F1C293D2AF759F01E125207D16C2AF2E
:100EFD00754301900129C290306202D292D2AF7532
:100F0D009F21E125C2AF754301900115C292306258
:100F1D0002D290D2AF759F01C26622900113757EE9
:100F2D0000C290C291C292D293D294D295C2622243
:100F3D00788076090876090876040876FF08760326
:100F4D000876FF08760B0876030876010876017897
:100F5D008C76010876FF0876FF0876FF0876FF0885
:100F6D0076FF0876030876FF0876FF0876FF087689
:100F7D00250876D00876280876500876040876FF7E
:100F8D0008760208760008767A0876FF087601085A
:100F9D007601087600087603227887E6FFC272BFD5
:100FAD000302D2727888E6C394036008C27DE630EE
:100FBD00E102D27DC27E7889E630E102D27EC3EFB6
:100FCD0094026008758E01D273020FDE758E00C219
:100FDD0073227880E6149000809378A4F67881E6E9
:100FED00149000809378A5F67886E61490008D9382
:100FFD0078A6F6789CE67538FF75390CB40206753F
:10100D0038A075390AB4030675388275390578A389
:10101D00E61490009A93F569120F2822227896E62D
:10102D00FA7897E6FB7888E6B40305C3EB940EFBDC
:10103D00307F047A007BFFC3EB9AFCC3948250028D
:10104D007C827575000575EC8575F0A4C3E5F0948B
:10105D007D40F222D27F112A1205A87A007B007CF6
:0E106D001012059EE55F2AFA74003BFBDCF3CF
:10107B007C04C3EB13FBEA13FADCF7FEC27F112AE5
:10108B0022E5EF20E6037520000520903FFFE520C9
:10109B00146006901DFF1460009304600375EF103D
:1010AB0053D9BF7581C043FF8012059975EF00437B
:1010BB00B203E5B3240420E70DF521E5E320E006B8
:1010CB008521B343E301120F287580FF75A40075CA
:1010DB00F19075D47F75903875A53F75F23F75D536
:1010EB000075A60175E241E4F8F6D8FD756B0112A7
:1010FB000F3D1215B878988676753001C2AF120580
:10110B00B21205C21205A81205C91205A81205D004
:10111B001205A8C2AF78FA79FA308707D9FBD8F74E
:10112B00021C00120FA6120FDF1129112A789886C4
:10113B0076120F2875885075891275C8247591041D
:10114B0075D84075A82275B80275E690759B8075A9
:10115B009D0075D10775BC5875BB0675BA1175E83E
:10116B0080120599D2AF1208A653DACF207E034323
:10117B00DA20307E0343DA1043DA01C2D8C271128F
:10118B0005B2D2617B037A0CE55E70077A0CDB0348
:10119B0002111E1205A820700302111EC270E55F1A
:1011AB00C3940240E1E52F541F856160F561B56082
:1011BB00D5DAD5C26153DACF207E0343DA20307EF5
:1011CB000343DA10C2D8C27178A2E67008D274E574
:1011DB002F54E0F52FC2757529001205AD30740937
:1011EB00C3E529940A4002D27512059E7802307429
:1011FB00027800C3E55F9840F0C2AF1205C212053A
:10120B00C21205C2D2AF1205B2754D007888E6B492
:10121B00030241F512059E788CE6C394015003023C
:10122B0012F5E530C3940150030212F5207435C357
:10123B00E55F94FF50030212F5C2AF1205D7D2AF90
:10124B001205ADC3E55F940150EFC2AF1205C21298
:10125B0005A31205C2D2AF1205ADC3E55F94FF40E3
:10126B00E90217607F02D27F112A1205ADC2AFC20D
:10127B007F112AAE5FC3E55F947FD2AF4076120534
:10128B0099C2AF1205D7D2AFDFDC1161C3EE940563
:10129B007897F61205B21215FA1216E37F0AD27F6F
:1012AB00112A1205ADC2AFC27F112AAE5FC3E55F33
:1012BB00947FD2AF50E6120599C2AF1205C2120548
:1012CB00A31205C2D2AFDFD61161EE24057896F6D4
:1012DB001205B21215FA1217121205AD112AC3E537
:1012EB005F94FF50024137021760C3E55F954D4095
:1012FB0003855F4D1205AD78017988E7B403027859
:10130B0005C3E55F9840024117C2AF1205D712051E
:10131B00D71205D7D2AF1205B2753000E4F531F50F
:10132B00320531E531F470390532789AE6781914C3
:10133B006012783214600D787D14600878FA1460AE
:10134B0003753200C3E53298401715327531B47806
:10135B00998676C2AF1205D7D2AF789886761205EA
:10136B00AD1205A3E52A7005307402211E78012009
:10137B0074027806C3E55F9840A77888E6C39403A8
:10138B0060031205ADE52A700302111EC2AF120FE6
:10139B0028E4F522F523F524F525F526F56AD2AFD9
:1013AB007885E6C333F568E4F545F546F547F5482A
:1013BB00F549F573F52CF52DF53775730875BB10DD
:1013CB001205991208AAE5E820ECFBA8BDA9BEE915
:1013DB007001F888741208AE75730875BB107887A6
:1013EB00E6FE7602120FA67887EEF6C2AF7564FFA3
:1013FB00120946852264852265852266D2AF752245
:10140B000175240175250175260185636C756D01C8
:10141B007888E6B40307C27D307602D27DD268D2DB
:10142B0069753300120E8E120EB312096612096D16
:10143B0012096612096D120966021454C2AF120F1B
:10144B00A6D2AF75730075BB06120BF11206A21272
:10145B000D0C120D5612096D120BE0306D031206B6
:0D146B00FE20670312084930670312089045
:10147800120D0C120D7B12096D120BF1306D031257
:101488000733120D0C120DF212096D120BE0306DBC
:1014980003120791120D0C120E1712096D120BF19F
:1014A800306D031207EE120D0C120E8E12096D121A
:1014B80008AA120BE0120D0C120EB31208AE120994
:1014C8006D306935206B3285676485676585636C27
:1014D800756D0179187A0CC3E53399400FC269D24A
:1014E8006A8A35856764856766021501C3E55F9476
:1014F80001400302145402157E306A1B206B18E564
:1015080035147004C26A8147F535C3E55F9401401C
:101518000302145402157E753600C3E56278FA9802
:101528005054307404E52A604D7888E6B4031720D7
:101538007D05207607A14E307602A14E206B07D29A
:101548006B856764819378F0306B058567647820D4
:10155800C3E5419850028154306B1BC26BC27D3089
:101568007602D27DD26A7535128567648154053654
:10157800E55F6002A181753600C2AF120F28788737
:10158800E6FE7602120FA67887EEF6E4F522F5233A
:10159800F524F525F526F568C268D2AF120599122B
:1015A8000F28307409C3E53694054002211E6127CF
:1015B800901A0D782012163CE520B4550CA312168B
:1015C8003CE520B4AA030215DA120F3D1215FA02FF
:1015D80015F9901A0378807B0A12163CA308DBF9E8
:1015E800901A0F788C7B1812163CA308DBF9901A16
:1015F8002722C2AF12167B121655901A00740E12CB
:101608001641A37404121641A37414121641901AB9
:101618000378807B0A121640A308DBF9901A0F782A
:101628008C7B18121640A308DBF912168E12166C62
:10163800901A2722E493F622E6438F01538FFD7513
:10164800EF0275B7A575B7F1F0538FFE22438F02ED
:10165800438F0175EF0275B7A575B7F1901A0DF0B4
:10166800538FFC22901A0D7455D141901A0E74AA0A
:10167800D141227A3079D07820901A40D13CE520A7
:10168800F709A3DAF7227A3079D0901A40E7D141E6
:1016980009A3DAF922AB77A878BB01027980BB02EB
:1016A800027981BB03027982BB04027984BB0502FB
:1016B8007986BB06027992BB07027987BB08027953
:1016C800A3BB0902799CBB0A027988BB0B02798902
:1016D800E8F7227C051205B2DCFB22C2AF1205C274
:1016E8001205C91205D01205D71205A31205C21298
:1016F80005C91205D01205D71205A31205C2120595
:10170800C91205D01205D7D2AF22C2AF1205D7121F
:1017180005D01205C91205C21205A31205D7120574
:10172800D01205C91205C21205A31205D71205D099
:101738001205C91205C2D2AF22AE77AF78C2AF1276
:1017480005C21205C21205C21205A3DEF21205D7A0
:101758001205A3DFF8D2AF22D1E3D1DBD1DB757755
:1017680001757801757900F1417C05AD5F1205B20C
:10177800C3ED955F70F5C3E55F9401400AC3E55F6B
:1017880094FF403202179CD19DB1FAD1E3C2AF75E4
:10179800EF10D1DBDCD50579C3E5799403500280DD
:1017A800C6D1DB0578E5771490009F93F808C3E568
:1017B8007898500280AED1DBD1DB0577C3E577940A
:1017C8000C5002809C120F3DB1FAC2AF75EF10D1D8
:0117D800DB35
:0319FD0002108C49
:101A00000E0414090904FF03FF0B03010155AA0189
:101A1000FFFFFFFFFF03FFFFFF25D0285004FF0259
:081A2000007AFF01010003FF41
:101A40002345415A5933417632232020202020203B
:101A500023424C48454C4923463333302320202031
:101A60002020202020202020202020202020202076
:101C0000C2AFC2D353D9BF7581C043B20343FF8073
:101C1000752438752503B1C975EF0275E24043F1AB
:101C20008053A47F75D400D2877DFA780379E67C4F
:101C300010752200752300901DD67B0675249875BB
:101C400025013087028142208708D8FBD9F9DCF7CB
:101C500081B4308708D8FBD9F9DCF781B4B189E4C5
:101C600093A3C39A6004DDC381B4DBDBB17B600264
:101C7000812B7B08E493FAA3B15CDBF87A30B15C8A
:101C8000752200752300B17BEAFCEBFDC3ED94FEE9
:101C9000400EB17B8A278B28ED30E0048A828B834B
:101CA000B17B7AC270D8C3ED94FE601350CEBD00F4
:101CB00025EC60097520007521FF0200008100A855
:101CC00027A9280809D804D90281D3B17FEA89AAB3
:101CD000F281C50D81A0C3ED94035049EDA2E092BD
:101CE000007AC5C3E5829400E583941C50902000DF
:101CF00010438F02438F0175B7A575B7F1F030001F
:101D00001FA827A9280809438F01538FFDD804D99C
:101D100002A12089AAE275B7A575B7F1F0A3A10DBC
:101D2000538FFC817C7AC1BD030CE493A3FAB140CC
:101D3000DCF8B138817C817EAA22AB23B15CEBFA5E
:101D4000EA6222752608C3E52313F523E52213F57D
:101D50002250066323A0632201D526EAB1C9B1C986
:101D600075260AEAF4200102D287300102C287B147
:101D7000C9C3134002C201D526EB22B17FEAFB2082
:101D80008702A17F308702A184752608AE24AF2583
:101D9000C3EF13FFEE13FEB1CDB1C9C3EA13308711
:101DA000024480FA30E703632201C3E52313F523DD
:101DB000E52213F52250066323A0632201D526D91C
:101DC000E52265236523F52222AE24AF250E0FDE22
:101DD000FEDFFCD20122424C48656C693437316326
:041DE000F3300601D5
:00000001FF
